:100000000C942D010C9455010C9455010C94550140
:100010000C9455010C9455010C9455010C94550108
:100020000C9455010C9455010C9430040C94540517
:100030000C9455010C9455010C9455010C945501E8
:100040000C9455010C9455010C9455010C945501D8
:100050000C9455010C9455010C9455010C946501B8
:100060000C9455010C9455010C9455010C945501B8
:100070000C9455010C9455010C9455010C945501A8
:100080000C9455010C9455010C9455010C94550198
:100090000C9455010C9455010C9455010C94550188
:1000A0000C9455010C9455010C945501050109025D
:1000B000A1010901A1008501050919012903150004
:1000C00025019503750181029501750581030501DF
:1000D0000930093109381581257F75089503810696
:1000E000C0C005010906A1018502050719E029E73D
:1000F0001500250175019508810295017508810398
:100100009506750815002565050719002965810004
:10011000C0090402000103000000092101010001DF
:100120002265000705840340000100000000000074
:1001300000002A2B28000000000000000000000042
:10014000000000000000000000002C9EB4A0A1A24E
:10015000A434A6A7A5AE362D3738271E1F2021228E
:1001600023242526B333B62EB7B89F848586878887
:10017000898A8B8C8D8E8F90919293949596979877
:10018000999A9B9C9D2F3130A3AD35040506070835
:10019000090A0B0C0D0E0F10111213141516171857
:1001A000191A1B1C1DAFB1B0B500040309042203CA
:1001B000410072006400750069006E006F0020004D
:1001C0004C0065006F006E006100720064006F00FB
:1001D0001803410072006400750069006E006F0032
:1001E00020004C004C0043001201000200000040BF
:1001F000412334000001010200011201000202004B
:1002000000404123340000010102000100C180814F
:10021000C1080B00020202010009040000010202F1
:100220000000052400100105240101010424020638
:1002300005240600010705810310004009040100A0
:10024000020A0000000705020240000007058302C1
:100250004000000075029504B60611241FBECFEFC2
:10026000DAE0DEBFCDBF11E0A0E0B1E0E6EEFEE0F7
:1002700002C005900D92A433B107D9F711E0A4E3B1
:10028000B1E001C01D92A935B107E1F712E0CAE55E
:10029000D2E004C02297FE010E946D07C435D10749
:1002A000C9F70E9420030C9471070C940000089574
:1002B0008EE391E060E071E00E94710368EE73E00C
:1002C00080E090E00E94AD0108951F920F920FB65A
:1002D0000F9211242F933F938F939F93AF93BF93CC
:1002E0008091380190913901A0913A01B0913B0180
:1002F00030913C010196A11DB11D232F2D5F2D379B
:1003000020F02D570196A11DB11D20933C01809333
:10031000380190933901A0933A01B0933B01809149
:10032000340190913501A0913601B09137010196C9
:10033000A11DB11D8093340190933501A093360126
:10034000B0933701BF91AF919F918F913F912F91C2
:100350000F900FBE0F901F9018959B01AC017FB7B7
:10036000F8948091340190913501A0913601B091BB
:10037000370166B5A89B05C06F3F19F00196A11D16
:10038000B11D7FBFBA2FA92F982F8827860F911DE7
:10039000A11DB11D62E0880F991FAA1FBB1F6A959E
:1003A000D1F7BC012DC0FFB7F89480913401909132
:1003B0003501A0913601B0913701E6B5A89B05C083
:1003C000EF3F19F00196A11DB11DFFBFBA2FA92F54
:1003D000982F88278E0F911DA11DB11DE2E0880F77
:1003E000991FAA1FBB1FEA95D1F7861B970B885E42
:1003F0009340C8F2215030404040504068517C4FFB
:10040000211531054105510571F60895789484B59B
:10041000826084BD84B5816084BD85B5826085BD00
:1004200085B5816085BDEEE6F0E0808181608083E6
:10043000E1E8F0E0108280818260808380818160C9
:100440008083E0E8F0E0808181608083E1EBF0E090
:10045000808184608083E0EBF0E080818160808334
:10046000E1E9F0E080818260808380818160808327
:10047000E0E9F0E0808181608083E1ECF0E0808160
:1004800082608083808181608083E0ECF0E0808105
:1004900081608083EAE7F0E08081846080838081EE
:1004A0008260808380818160808380818068808396
:1004B0000895FC0191818081813A31F4913089F075
:1004C00080E0933089F40DC0813269F49B3021F4CF
:1004D000828180930F0105C09A3029F48281809334
:1004E000100181E0089580E0089510923D0110927E
:1004F0004101109240018FE191E090933F01809380
:100500003E0110924301109242010895EF92FF9232
:100510000F931F93DF93CF930F92CDB7DEB78983ED
:100520008B017A0184E0BE016F5F7F4F41E050E0B4
:100530000E94960484E4B801A7010E9496040F90DB
:10054000CF91DF911F910F91FF90EF90089582E07E
:1005500048E050E00E9486020895EF92FF920F93C8
:100560001F93DF93CF93CDB7DEB728970FB6F894DC
:10057000DEBF0FBECDBF7C019E012F5F3F4F88E0E5
:10058000F90111928A95E9F7F701A481B5811097D5
:1005900059F0ED91FC9111970190F081E02DCD0182
:1005A00070E0A901099518C067FD07C0E62FF0E0CB
:1005B000E65DFE4F6491662341F481E090E0F7012F
:1005C0009383828320E030E019C067FF04C08981F3
:1005D000826089836F776B83C7018E010F5F1F4F26
:1005E000B8010E94A70288E0F80111928A95E9F704
:1005F000C701B8010E94A70221E030E0C901289696
:100600000FB6F894DEBF0FBECDBFCF91DF911F9123
:100610000F91FF90EF90089580E86CEA70E045E656
:1006200050E00E94CA030895FC0180818F5F80839F
:1006300080E861E171E049E150E00E94CA03089559
:10064000CF93DF930E9406028CE491E00E947C0429
:100650000E945701C0E0D0E00E9458012097E1F3CA
:100660000E940000F9CFCF92DF92EF92FF920F939A
:100670001F93CF93DF937C016B018A01C0E0D0E030
:100680000FC0D6016D916D01D701ED91FC910190E4
:10069000F081E02DC7010995C80FD91F0150104006
:1006A0000115110571F7CE01DF91CF911F910F91C7
:1006B000FF90EF90DF90CF900895CF93DF93DB0111
:1006C0000D900020E9F71197A61BB70BEC01E8810C
:1006D000F9810280F381E02DAD010995DF91CF9181
:1006E00008950E945D0308959FB7F89487708093E2
:1006F000E9008091F2009FBF0895282F8091460164
:100700008823C1F057FF1AC015C02898909345015F
:100710008091F1008193E217F307B9F74115510574
:1007200039F08091F200882319F48BE68093E80079
:10073000AFBF02C04FEF5FEFCA010895AFB7F894A3
:1007400027702093E9008091F200282F30E02417D1
:1007500035070CF4A901FB019B01240F311D94E620
:10076000DACFDF93CF930F92CDB7DEB7BE016F5FC5
:100770007F4F41E050E00E947D03019719F02FEF79
:100780003FEF03C08981282F30E0C9010F90CF913E
:10079000DF910895FF920F931F93F82E142F052FCA
:1007A0004091490150914A01212F302FC901DC01AC
:1007B000FB016EEF29C0F7FE02C0949101C0908149
:1007C000209147013091480124173507ACF48091FE
:1007D000E8008570E1F38091E80082FF03C02FEF0D
:1007E0003FEF17C09093F100C90101968F7390708D
:1007F000892B11F46093E8002F5F3F4F309348013D
:1008000020934701119731961097A9F6812F902FC9
:100810009C01C9011F910F91FF9008959C01809147
:10082000E80082FFFCCFF901260F311D03C0809143
:10083000F1008193E217F307D1F7289884E68093BB
:1008400045018BEF8093E800CB0108958093E90088
:100850008091F200882319F08AE38093E8000895DC
:100860001F920F920FB60F9211248F939F93809136
:10087000E1001092E100982F83FF0FC01092E90071
:1008800081E08093EB001092EC0082E38093ED0016
:100890001092460188E08093F00092FF26C083E02A
:1008A0008093E9008091F200882319F08AE3809315
:1008B000E80080914401882351F0809144018150E7
:1008C0008093440180914401882309F45D9A8091CA
:1008D0004501882351F08091450181508093450165
:1008E00080914501882309F4289A9F918F910F9058
:1008F0000FBE0F901F9018951092460181E08093D3
:10090000D70080EA8093D80082E189BD09B400FE57
:10091000FDCF80E98093D8008CE08093E2001092B4
:10092000E000559A209A0895089508955F926F9275
:100930007F928F929F92AF92BF92CF92DF92EF926F
:10094000FF920F931F93CF93DF93E82E842E752E83
:1009500080914601882371F18B01242F352FC90125
:10096000EC017AEFF72E67E0962E9E2050E4552E8C
:100970008E2D90E040E2A42EB12CA822B9223AE3B9
:10098000632E20E4C22ED12CC822D92258C09FB792
:10099000F8949092E9008091E80085FD02C020E083
:1009A00004C08091F200252D281B9FBF222361F4F3
:1009B000FA9419F42FEF3FEF4DC061E070E080E052
:1009C00090E00E94AD013BC0822F90E0C817D9078C
:1009D0000CF42C2FC21BD1094FB7F8949092E90068
:1009E000A114B10421F406C01092F1002150222379
:1009F000D9F719C0E7FC03C0F801922F10C0C80155
:100A0000322F06C0FC010196E491E093F1003150D1
:100A10003323C1F706C081918093F100915099234F
:100A2000D1F7020F111D8091E80085FF05C02097C6
:100A300029F4C114D10411F06092E8004FBF20974F
:100A400009F0A5CF5D9884E680934401282D372DC9
:100A5000C9019C01C901DF91CF911F910F91FF90B6
:100A6000EF90DF90CF90BF90AF909F908F907F904E
:100A70006F905F9008950F931F93DF93CF930F9222
:100A8000CDB7DEB719828E010F5F1F4FC8010E94DC
:100A90001D07C8010E941403898190E00F90CF9137
:100AA000DF911F910F9108951F920F920FB60F9231
:100AB0001124EF92FF921F932F933F934F935F93D5
:100AC0006F937F938F939F93AF93BF93EF93FF9316
:100AD000DF93CF93CDB7DEB76197DEBFCDBF109266
:100AE000E9008091E80083FF0FC1FE0131969E016D
:100AF000275F3F4F03C08091F1008193E217F30716
:100B0000D1F7289884E68093450182EF8093E8002E
:100B1000998197FF05C08091E80080FFFCCF03C05A
:100B20008EEF8093E800292F30E0C9018076907025
:100B3000892B09F0C2C08A81882329F41092F10020
:100B40001092F100D6C0813009F4D3C0833009F48B
:100B5000D0C0853049F48091E80080FFFCCF8B81C4
:100B600080688093E300C5C0863009F07CC01C819A
:100B7000EF80F8841230C1F51092E900109248011C
:100B80001092470110924A01109249010E943B05C0
:100B900099E0FE013996DF01292F1D922A95E9F788
:100BA00099871A8791E09E8790E8988B9AEF998BA6
:100BB0002091470130914801275F3F4F3C872B87A9
:100BC0008D871092E9001092480110924701F0922F
:100BD0004A01E092490180E0BF0149E050E00E94F3
:100BE000CA030E943B0585C01092E900109248019B
:100BF00010924701F0924A01E0924901123241F409
:100C000082E290E00E940C03892B09F476C071C047
:100C1000113079F488E0E816F10419F481E080934A
:100C20004B0180914B01882309F06BC0E8EEF1E0A5
:100C300013C0133009F061C08B81882319F4EAEAEC
:100C4000F1E00AC0823019F4EEEAF1E005C081302B
:100C500009F053C0E0EDF1E0449180E8BF0150E0BD
:100C60000E94CA0346C0873009F447C0883021F487
:100C700081E08093F1003DC08930D9F52370307058
:100C8000232BD9F5EDE0F2E091E031E026E39093FB
:100C9000E9003093EB0084918093EC002093ED0009
:100CA0009F5F3196953099F78EE78093EA00109216
:100CB000EA008B81809346011CC08F819885109239
:100CC000E900109248011092470190934A018093E5
:100CD00049018D81882329F4CE0101960E943107B4
:100CE00006C0823051F4CE0101960E945902882339
:100CF00021F08EEF8093E80007C081E28093EB0043
:100D000003C0EAEFF1E0A8CF6196DEBFCDBFCF917F
:100D1000DF91FF91EF91BF91AF919F918F917F9163
:100D20006F915F914F913F912F911F91FF90EF90A5
:100D30000F900FBE0F901F901895DC01809111014C
:100D4000909112018F5F9F4F61F4ED91FC9111978B
:100D50000680F781E02DCD010995909312018093D3
:100D6000110180911101909112010895109250018A
:100D700010924F0188EE93E0A0E0B0E08093510123
:100D800090935201A0935301B093540187E291E0F4
:100D900090934E0180934D0108950F931F93DF931D
:100DA000CF930F92CDB7DEB78C01698380911A0182
:100DB000882369F083E0BE016F5F7F4F41E050E020
:100DC0000E9496041816190614F49C0107C081E0CD
:100DD00090E0F8019383828320E030E0C9010F9016
:100DE000CF91DF911F910F91089583E00E94260417
:100DF000089520911101309112018FEF2F3F380794
:100E000039F08FEF9FEF909312018093110104C08E
:100E100082E00E94B1039C01C901089582E00E9412
:100E20007403282F80911101909112018F5F9F4FC1
:100E300009F02F5F822F90E00895FC0180818E5F82
:100E4000808380E861E172E042E450E00E94CA03DE
:100E500008958CE491E00E949404F8940C94003C72
:100E60000895CF93DF93EC0189819881913A51F4F1
:100E7000813269F580E063E171E047E050E00E9473
:100E8000CA0323C0913219F5803239F483E191E02D
:100E900067E070E00E940E0418C08232C1F48091B5
:100EA0001A01882379F08091130190911401A09187
:100EB0001501B0911601805B9440A040B04011F440
:100EC0000E9429078A8180931A0181E001C080E095
:100ED000DF91CF910895EE0FFF1F0590F491E02D63
:060EE0000994F894FFCF15
:100EE60048656C6C6F2041726475696E6F200001F5
:100EF60001FFFF00E100000000000000000000AD5F
:100F060002330300000000CD0633030E07F9069DE9
:040F160006F50600D6
:00000001FF
